:0401AC00AA82AB83F5
:0E01B0008A828B83E493FCA3AA82AB83ECFDCE
:0E01BE00600F8D82C002C00312149FD003D0C8
:0301CC000280E1CD
:0101CF00220D
:0601D0009040C40201ACE6
:0B01D60012158AE58260069040C812F6
:0201E10001AC6F
:0401E3007808E4F2C2
:0D01E70012150A121538AA82BA0802800308
:0301F400BA7F16B9
:0C01F7007808E260EB12158AE5826003D4
:030203001201D015
:070206007808E214F280DA2F
:03020D00BA151609
:0C0210007808E260D212158AE5826003D3
:03021C001201D0FC
:07021F007808E214F280EA06
:05022600BA0D027A0A86
:0E022B00BA0A0F12158AE582603775820A1230
:04023900149F802F5F
:06023D007808E2B42E0077
:0A02430050A27808E2FB780804F2EC
:0A024D00EB2434F582E434F0F5836D
:0E025700EAF0C00212158AE582D00260838AA6
:070265008212149F0201E761
:0A026C007808E2FA780804F2EA24A8
:0A02760034F582E434F0F583740AD5
:0A028000F07808E2FA780804F2EAC8
:0A028A002434F582E434F0F583E437
:06029400F07809E4F222FB
:08029A007806740AF278097974
:0B02A20008C3E3F5F0E295F050177878
:0902AD0009E2FA780904F2EA24DE
:0A02B60034F582E434F0F583E0FA39
:0302C0007806F2CB
:0102C3002218
:0502C400AA82BA0A0045
:0A02C900500874302AF58202149FD9
:0802D30074572AF58202149F02
:0E02DB00121538AA82C3EA648094B0401174F0
:0E02E900B98AF063F08095F04006EA24D0F563
:0202F700822261
:0E02F900C3EA648094E1401174E68AF063F079
:0B0307008095F04006EA24A9F5822250
:0E031200C3EA648094C1401174C68AF063F09F
:0B0320008095F04006EA24C9F5822217
:09032B0078077401F275820022CA
:0E033400AA82AB838B82C002C00312034AD0A0
:0803420003D0028A8202034A83
:0E034A00E582FAC4540FFB740F5BF582C0020B
:0D0358001202C4D002740F5AF5820202C4D2
:080365007806E2B42002800CCE
:08036D007806E2B409028004E5
:040375007A00800288
:020379007A0107
:03037B008A822251
:0C037E00120365E582600512029A80F40B
:01038A002250
:0E038B00AA82C3EA648094B0401174B98AF06B
:0D03990063F08095F04006EA24D0F5822242
:0E03A600C3EA648094E1401174E68AF063F0CB
:0B03B4008095F0400674A92AF5822213
:0E03BF00C3EA648094C1401174C68AF063F0F2
:0B03CD008095F0400674C92AF58222DA
:0403D8007582FF2209
:0B03DC007800E4F208F212037E7A00C1
:0303E700BA020057
:0C03EA0050477806E2F582C00212038B37
:0C03F600AB82D002EB30E70678077402FF
:02040200F222E4
:0C0404007800E2FC08E2C454F0CCC4CC48
:0E0410006CCC54F0CC6CFDEB3395E0FEEB426F
:0C041E0004EE42057800ECF208EDF2C09C
:09042A000212029AD0020A80B409
:0104330022A6
:0B0434007A017800E4F208F2C0021226
:04043F00037ED00266
:0C0443007806E2F582C00212038BAB8247
:0C044F00D002EB20E7307800E2FC08E26D
:0E045B00C454F0CCC4CC6CCC54F0CC6CFDEB93
:0C0469003395E0FEEB4204EE4205780003
:0E047500ECF208EDF27A00C00212029AD002F8
:0204830080BE39
:07048500EA60047807EAF2C7
:01048C00224D
:0A048D00C01FE581F51F2404F5816E
:0C0497007A017802E4F208F208F208F2A0
:0704A300C00212037ED0022B
:0B04AA007806C3E2648094B0500302A7
:0204B500052E12
:0C04B7007806C3E2F5F074B963F080959C
:0A04C300F040687802E2F54F08E20D
:0904CD00F55008E2F55108E2F5D2
:0B04D6005290000AE4F5F0123966A80D
:0C04E1001F08A68208A68308A6F008F6F3
:0C04ED007806E2FFE23395E0FBEF24D03C
:0C04F900FFEB34FFFB3395E0FCFDA81F77
:0E05050008EF26FFEB0836FBEC0836FCED088D
:0C05130036FD7802EFF208EBF208ECF283
:0D051F0008EDF27A00C00212029AD002022A
:02052C0004AA1F
:07052E00EA60047807EAF21D
:0A05350078027900E2F308E209F30E
:06053F00851F81D01F2280
:04054500AA82AB8358
:0C0549008A828B83E493FC60237806E236
:05055500B5040280095D
:09055A0078077402F27582002298
:050563000ABA00010BC3
:0D056800C002C00312029AD003D00280D45A
:040575007582012268
:090579001204347807E2704678A0
:0C0582000FC2D575F007E230E704B2D5D7
:02058E00F40473
:0E059000A430D50AF42401C5F0F43400C5F0FF
:0A059E0024ADFA74F335F0FB740687
:0C05A8002AF582E43BF5837800E2B40001
:0A05B4000908E2B40004740180019C
:0105BE00E458
:0405BF00FAB4010089
:0405C300E433FAF033
:0105C7002211
:0705C80012037E9040CB12EC
:0705CF000545E582700122E1
:0D05D60012150A90006412191175C90B90DE
:0B05E30000C8121911758208021411E3
:0D05EE009000A4E493C0E0740193C0E07499
:0A05FB0012C0E07448C0E07480C034
:0A060500E07402C0E07448C0E07425
:0A060F0080C0E074D1C0E07440C068
:0E061900E07480C0E0123A70E58124F5F581AE
:0A06270074FAC0E07447C0E074806C
:0A063100C0E0740EC0E07441C0E0A8
:0E063B007480C0E0123A70E58124FAF5812245
:04064900780BE4F254
:0A064D00780B790AC3E3F5F0E2959B
:04065700F04001224C
:0A065B00780BE225E02464F582E448
:0A06650034F0F583E0FBA3E0FC781D
:03066F000CE4F2A6
:0C067200780CE275F004A4FEAFF02BF54C
:0E067E0082EF3CF583E493FAA3E493FD4A7007
:04068C000302071945
:0E069000EE2BFEEF3CFF8E828F83A3A3E4933C
:08069E00F508A3E493F50985BA
:0A06A6000882850983C003C0041216
:0506B00001ACAE08AF33
:0C06B500097A808E828F838AF012401E2A
:0E06C100AA82D004D0038A057E000DBD000180
:0106CF000E1C
:0706D000ED2508F508EE35E9
:0806D70009F509742DC39AFA1C
:0E06DF008A051AED6014758220C002C003C0A7
:0C06ED000412149FD004D003D00280E659
:0A06F900850882850983C003C00450
:0E0703001201AC75820A12149FD004D0037844
:080711000CE22401F202067261
:09071900780BE22401F202064D06
:080722007807E2B40102800631
:06072A007807E2B4020DA5
:0A07300090412375F0801239FD7826
:03073A0007E4F2DF
:01073D002299
:0A073E00AA82AB83780AE2B40B0034
:0E074800400E758206C002C003121411D003C9
:02075600D002CF
:0A075800780AE2FC780A04F2EC2CA7
:0A0762002464F582E434F0F583EA24
:05076C00F0A3EBF022F8
:070771001201D612029A12D8
:09077800037E7806E2FAC00212C9
:09078100029AD002BA0D0280E7D1
:05078A00BA0A0280E242
:0A078F0090F07AE4F0A3F0750A0080
:0A079900780AC3E2F5F0E50A95F0D6
:0507A3004003020825DF
:0507A800E50A250A240A
:0A07AD0064F582E434F0F583E0FC0B
:0507B700A3E0FD7E003F
:0A07BC00EE75F004A4F50B85F00CB7
:0C07C6002CF582E50C3DF583E493FFA3C5
:0B07D200E493FB4F603DE50B2CFBE5C2
:0C07DD000C3DFF8B828F83A3A3E493FBF1
:0E07E900A3E493FF8B828F83E493FBB5021B86
:0A07F700E50B2CF582E50C3DF583BF
:0E080100E493FBA3E493FF90F07AEBF0A3EFF7
:03080F00F0800373
:030812000E80A7AE
:0C08150090F07AE0FBA3E0FC4B700505BE
:040821000A02079927
:0E08250090F07AE0FAA3E0FB4A6011C002C036
:0E083300038A828B8312008BD003D0028005D3
:0508410078077402F2CB
:06084600120722020771F7
:07084C0090413012073E74D9
:0808530048C0E07441C0E074EC
:08085B0071C0E07407C0E090D9
:0C086300F07C12161DE58124FCF58122BA
:0440C40008200800C8
:0340C8003E200097
:0640CB0065626F6F7400D6
:0E40D1006D616E756661637475726572202094
:0E40DF0020202025730A70726F6475637420B0
:0E40ED0020202020202020202025730A73652B
:0E40FB007269616C2D6E756D626572202020F9
:054109002025750A00ED
:0E410E00736F6674776172652D7665727369E2
:07411C006F6E2025730A00FD
:0D41230053796E746178206572726F7200BE
:0241300049063E
:024132004C41FE
:024134005D1913
:024136005341F3
:02413800790507
:02413A005B41E7
:02413C00C805B4
:02413E007041CE
:02414000EE058A
:064142007F4100000000B7
:04414800636D64003F
:07414C003F0048656C7000A4
:0841530054005461736B73000A
:0E415B0045203C30206F66662C2031206F6EB0
:074169003E004563686F0092
:0E417000722065626F6F74005265626F6F742B
:01417E000040
:0A417F00760056657273696F6E00DA
:0E086F0090F106E0FAA3E0FBA3E0FCA3E0FD9D
:0E087D0090F125E0FEA3E0FFA3E0F8A3E0F970
:0E088B00C002C003C004C0058E828F8388F0B7
:0E089900E91219C0AA82AB83ACF0FDE5812400
:0E08A700FCF58190F110EAF0A3EBF0A3ECF069
:0408B500A3EDF0229D
:0608B900780DE26001224F
:0A08BF0090F0F3E0FABA0102803C69
:0C08C90090F0F37401F090F0F4E4F09073
:0C08D500F0F574FAF0A3E4F0754F007524
:0608E1005009E4F55190FE
:0608E700F0FA122DD47A94
:0408ED00897B418A38
:0408F1004F8B507564
:0608F5005106E4F55290EB
:0608FB00F0FA122D9F909F
:04090100F0F9E4F035
:0B09050090F0F4E0FABA15030209E9D3
:03091000BA010029
:07091300500590F103E4F030
:03091A00BA02001E
:0E091D00500E90F0F7E4F0A3F090F104E4F037
:02092B00A3F037
:03092D00BA03000A
:0E09300050209000A6E493FB740193FC740227
:0E093E0093FD740393FE90F106EBF0A3ECF032
:06094C00A3EDF0A3EEF0A4
:03095200BA0500E3
:07095500500590F10EE4F0E3
:03095C00BA0600D8
:07095F00500590F10FE4F0D8
:03096600BA0800CC
:08096900500690F1147401F036
:03097100BA0900C0
:0A0974005013754F00755010E4F5A4
:07097E005190F115C00212B7
:040985002DD4D0029B
:03098900BA0A00A7
:0E098C00502E90F0F9E075F064A4FBE5F0FC4D
:0E099A003395E0FDFE74762BFB74A13CFC74DB
:0E09A800063DFDE43EFE90F125EBF0A3ECF0E1
:0609B600A3EDF0A3EEF03A
:0309BC00BA0B0073
:0909BF00500790F129E4F0A3F0C7
:0309C800BA0D0065
:0909CB00500790F12BE4F0A3F0B9
:0309D400BA140052
:0709D700500590F12DE4F042
:0B09DE0090F0F47415F0780E7401F234
:0909E90012086F780D7401F2226E
:0709F20090F12E12135102D7
:0209F90008B93B
:0909FB00780E7401F290F12E0255
:020A040013AF2E
:070A06001209F290F12E022B
:020A0D0013AF25
:0A0A0F0074FAC0E074F0C0E0E4C027
:0A0A1900E07490C0E07441C0E07486
:0D0A230080C0E0123A70E58124FAF58122CE
:080A3000754F00755009E4F553
:050A38005190F12F12A6
:070A3D002DD412037E7A00A4
:080A44007806E2B40A028026E4
:030A4C00BA0800E5
:0C0A4F0050138A030AEB242FF582E434D4
:090A5B00F1F5837806E2F0800554
:050A640078077401F2A7
:090A6900C00212029AD00280D2F0
:060A72007807E26001229A
:050A78001209F2754FA8
:030A7D002F755082
:060A8000F1755109E4F5D7
:050A86005290F0FA128D
:050A8B002D9F0209FB94
:0E0A900090F125E0FAA3E0FBA3E0FCA3E0FD5B
:0C0A9E00C002C003C004C00574A0C0E08A
:0C0AAA007441C0E07480C0E0123A70E5B6
:060AB6008124F9F5812204
:090ABC0012048D7807E2600122AA
:070AC5001209F290F12578FF
:0C0ACC0002E2F0A308E2F0A308E2F0A3AD
:0A0AD80008E2F012086F1209FB0299
:020AE20028F1F9
:0E0AE40090F106E0FAA3E0FBA3E0FCA3E0FD26
:0C0AF200C002C003C004C00574B0C0E026
:0C0AFE007441C0E07480C0E0123A70E562
:060B0A008124F9F58122AF
:090B100012048D7807E260012255
:070B19001209F290F10678C9
:0C0B200002E2F0A308E2F0A308E2F0A358
:090B2C0008E2F012086F0209FB57
:0C0B350090F12DE0FA7B00C002C00374B8
:0A0B4100C0C0E07441C0E07480C041
:0B0B4B00E0123A70E58124FBF58122E6
:090B560012048D7807E26001220F
:0C0B5F007800C3E2F5F0740295F008E2A3
:0C0B6B00F5F0E495F0500678077401F2F4
:010B7700225B
:070B78001209F27800E2907F
:070B7F00F12DF01209FB0249
:020B860028F154
:0C0B880090F114E0FA7B00C002C003747E
:0A0B9400D4C0E07441C0E07480C0DA
:0B0B9E00E0123A70E58124FBF5812293
:090BA90012048D7807E2600122BC
:070BB2001209F27800E29045
:060BB900F114F00209FB3B
:0A0BBF0012037E7806E2FAC002126B
:060BC900029AD0027B003D
:0E0BCF00EB75F006A4FCFD9041E693CDA393D8
:090BDD00FEBD0005BE00028032DD
:0C0BE6008D828E83E493FDB50225EC2483
:0A0BF200E6FCE43441FD8C828D83A3
:0E0BFC00A3A3E493FCA3E493FDC004C0058C06
:0B0C0A00828D8312008BD005D00422E5
:030C15000B80B79A
:060C180078077402F222CD
:020C1E007A005A
:0E0C2000EA75F006A4FBFC9041E693CCA3938A
:080C2E00FDBC0004BD00012221
:0E0C360074012CFEE43DFF78808C828D838853
:0E0C4400F0C002C003C006C00712401EAC8202
:0E0C5200AD83D007D006D003EC2EFEED3FFFA1
:0E0C60007C80EB9041E693CBA393FD7880C09F
:0C0C6E0006C007C004C003C005C000742D
:0A0C7A0016C0E07442C0E07480C0B0
:0E0C8400E0123A70E58124F7F581D0020A02F1
:020C92000C2034
:0B0C9400120A0690F0F4E0FA7B0090DA
:0E0C9F00F0F3E0FC7D00C002C003C004C005FD
:0A0CAD007420C0E07442C0E07480BF
:0D0CB700C0E0123A70E58124F9F5817A0061
:0E0CC400EA75F006A4FBFC9041E693CCA393E6
:080CD200FDBC0004BD0001227D
:0A0CDA00EB24E6FBE43441FC8B82BE
:0E0CE4008C83A3A3A3A3E493FBA3E493FC4B94
:0D0CF2006013C002C003C0048B828C83120B
:080CFF00008BD004D003D002E9
:030D07000A80BAA5
:060D0A0090423702073E93
:074189004E3043414C4C0095
:0E41900043616C6C7369676E3A2022257322BE
:02419E000A0015
:0E41A0004672657175656E63793A20256C6410
:0241AE000A0005
:0E41B000526164696F2063616C3A20256C6473
:0241BE000A00F5
:0E41C00054656C656D6574727920726174656A
:0641CE003A2025640A00FE
:0E41D400526164696F20656E61626C653A200D
:0441E20025640A0046
:0241E6003F4256
:0241E800BC0A0F
:0241EA00900A39
:0241EC00584237
:0241EE00300A95
:0241F0000F0AB4
:0241F200774212
:0241F400A90B15
:0241F600880B34
:0241F800A842DB
:0241FA00100BA8
:0241FC00E40AD3
:0241FE00D342AA
:02420000560B5B
:02420200350B7A
:02420400024373
:04420600940C000014
:02420A00094366
:0A420C001E0C00000000000000007E
:0A421600252D3230732025730A00B5
:0E422000436F6E6669672076657273696F6E14
:09422E003A2025642E25640A00E3
:02423700BF0BBB
:064239001043000000002C
:0E423F0046203C667265713E004672657175E0
:0B424D00656E637920286B487A290019
:0E42580063203C63616C6C3E0043616C6C73D0
:0E42660069676E2028382063686172206D61E0
:03427400782900A6
:0E42770065203C302064697361626C652C2008
:0E4285003120656E61626C653E00456E6162BF
:0E4293006C652074656C656D657472792061D0
:0742A1006E64205244460048
:0E42A80066203C63616C3E00526164696F20C9
:0E42B60063616C6962202863616C203D207298
:0E42C400662F287874616C2F325E31362929FE
:0142D20000EB
:0E42D30054203C726174653E0054656C656D4C
:0E42E1006574727920726174652028303D3357
:0E42EF00382E342C20313D392E362C20323D15
:0542FD00322E342900FF
:07430200730053686F7700A0
:074309003F0048656C7000E5
:0E43100063203C7661723E203C76616C7565E0
:0E431E003E0053657420636F6E666967202849
:0E432C003F20666F722068656C702C20732035
:09433A00746F2073686F7729008D
:0A0D1000C01F85811FC082C083E56B
:0C0D1A00812408F581A81F08740626FC3F
:0E0D2600E40836FD8C828D83E0FE30E4047F0D
:030D34006C800AC6
:080D3700EE30E5047F75800237
:020D3F007F65CE
:0E0D410053060F7A00EF3395E0FBC004C005A7
:0C0D4F00C006C002C007C0037443C0E02F
:0C0D5B007443C0E07480C0E0123A70E500
:0E0D67008124F9F581D005D0048C828D83E0C3
:070D7500FA20E403020FB8AD
:0C0D7C00A81F08740F26F582E40836F565
:0C0D880083A81F080808E0F6A3E008F6A6
:0C0D9400A81F08740B26F582E40836F551
:0C0DA00083E51F2405F8E0F6A3E008F648
:0C0DAC00A3E008F6A3E008F6A81F0874F6
:0E0DB8000726F582E40836F583E0FAA3E0FB97
:0C0DC600A3E0FEA3E0FFC004C005A81FCE
:0C0DD200080808E6C0E008E6C0E0E51FE5
:0E0DDE002405F8E6C0E008E6C0E008E6C0E044
:0D0DEC0008E6C0E0C002C003C006C00774E6
:0A0DF90050C0E07443C0E07480C0F5
:0E0E0300E0123A70E58124F3F581D005D004A9
:0E0E11008C828D83E0FA30E658C004C005A83C
:0C0E1F001F088682088683A3A3E0FA7BEC
:0C0E2B0000A81F088682088683A3E0FE52
:0C0E37007F00A81F088682088683E0FC6C
:0E0E43007D00C004C005C002C003C006C00789
:0A0E5100C004C005746AC0E07443D9
:0E0E5B00C0E07480C0E0123A70E58124F7F523
:090E690081D005D004D005D004AD
:0C0E7200A81F088682088683A3A3A3A300
:0C0E7E00A3E0FA7B00A81F08868208860B
:0C0E8A0083A3A3A3A3E0FEE51F2405F84A
:0C0E9600A606087600A81F0886820886C1
:0E0EA20083A3A3A3E0FE7F00C004C005C0022E
:0C0EB000C003E51F2405F8E6C0E008E6DA
:0B0EBC00C0E0C006C0077480C0E074F6
:0C0EC70043C0E07480C0E0123A70E58186
:0C0ED30024F7F581A81F08741426F5828E
:0E0EDF00E40836F583E075F002A4FAABF0C02B
:0A0EED0002C0037496C0E07443C015
:0E0EF700E07480C0E0123A70E58124FBF581C2
:0E0F0500D005D0048C828D83E0FC20E703022F
:020F13000FB815
:0C0F1500A81F08741326F582E40836F5C6
:0C0F210083E0FAE4CA25E0CA33FBA81FF5
:0E0F2D0008741126F582E40836F583E0FCA373
:0C0F3B00E0FDA81F08741526F582E408EC
:0C0F470036F583E51F2405F8E0F6A3E072
:0C0F530008F6A81F08741926F582E408AF
:0C0F5F0036F583A81F080808E0F6A3E0A0
:0C0F6B0008F6A81F08741726F582E40899
:0E0F770036F583E0FEA3E0FFC002C003C00415
:0C0F8500C005E51F2405F8E6C0E008E602
:0C0F9100C0E0A81F080808E6C0E008E661
:0B0F9D00C0E0C006C007749FC0E074F5
:0C0FA80043C0E07480C0E0123A70E581A4
:040FB40024F3F581AC
:060FB800851F81D01F22FD
:0A0FBE00C01FE581F51F2404F58132
:0C0FC800AA82AB83E0FCA81F08A604A8C6
:080FD4001F08E670030210C0C3
:0C0FDC0074012AFCE43BFFA81F08087603
:070FE800008C058F067F005D
:0C0FEF00A81F08C3EF9650168D828E8359
:080FFB00E06005A81F080806CC
:0A10030074022DFDE43EFE0F80E2B2
:0C100D00A81F080886077D00C002C00371
:0A101900C007C00574C5C0E07443B1
:0E102300C0E07480C0E0123A70E58124FBF555
:0D10310081D003D00274012AFCE43BFFA82B
:0B103E001F080876008C038F057E0061
:0C104900A81F08C3EE96506F8B828D83A9
:0E105500E0FF605DC0068B828D83A3E0FEA8E5
:0A1063001F080808A606087600A87A
:0C106D001F080886047A007E00C003C043
:0C10790005C006A81F080808E6C0E00833
:0E108500E6C0E0C004C002C007C006C004C040
:0A1093000274CDC0E07443C0E074A5
:0E109D0080C0E0123A70E58124F5F581D0069E
:0B10AB00D005D003A81F080806D006DF
:0A10B60074022BFBE43DFD0E80895F
:0610C000851F81D01F22F4
:0D4343006720256320675F6E202564200041
:0E435000675F6E7320256C6420675F657720C1
:0C435E00256C6420675F6120256420004E
:0E436A00675F5920256420675F4D2025642081
:08437800675F4420256420006A
:0E438000675F6820256420675F6D202564203C
:08438E00675F73202564200025
:09439600675F68642025642000C3
:0E439F00675F686520256420675F76652025CE
:0E43AD006420675F7620256420675F67202507
:0A43BB006420675F63202564200082
:0843C500735F6E2025642000E7
:0E43CD00735F76256420256420735F6325648A
:0543DB00202564200014
:0710C600E50D60031228F1A3
:0910CD00E50E6005750D00800CB4
:0610D600E5106005851025
:0310DC000D800381
:0310DF00850F0D6D
:0B10E2007A0D7BFF8A828B8302187F4F
:0A10ED00E4B50D0D7A0D7BFF8A8239
:0710F7008B8312184180EF0A
:0910FE00E50D24DF5003750D20FF
:0A1107007402250DFAE51175F022BF
:0A111100A42438F58274F135F0F5DE
:0E111B0083E4C0E0C0021227E2AA821581150B
:0A11290081EA60C0E511045407F5E7
:0A113300117A117BFF8A828B831270
:04113D00187F80ACEB
:0C1141007A117BFF8A828B8312184174A4
:0E114D000AC0E0E4C0E075820112221F158185
:04115B00158180E298
:02115F00AA11D3
:0A116100E51070117B107CFF8B82FB
:0B116B008C83C002121841D00280EB00
:09117600EAB51115E51060117BCA
:0C117F00117CFF8B828C83C0021218418F
:04118B00D00280E727
:0A118F00E51060CEEA75F022A424FA
:0411990038F512749F
:0A119D00F135F0F513EA045407FAE7
:0711A700E4B50D0302127113
:0A11AE00C00274F0C0E07443C0E01A
:0E11B8007480C0E0123A7015811581158174A3
:0C11C60002250DC4540F9043E093F58205
:0A11D20012149F7402250D540F90B3
:0E11DC0043E093F58212149FD0027D5A7E00EC
:0C11EA00AF0D780074022FFFE438F88E7F
:0E11F600017B00C3E99FEB648088F063F0800A
:0B12040095F05042EE2512F582E43513
:0C120F0013F583E0FB2DFDEBC4540F90A1
:0E121B0043E093F582C002C003C005C0061276
:0E122900149FD006D005D003740F5B9043E0F5
:0E12370093F582C005C00612149FD006D005A4
:05124500D0020E80A0A4
:0E124A00EDC4540F9043E093F582C002C0053E
:0E12580012149FD005740F5D9043E093F58251
:0B12660012149F75820A12149FD00220
:0A127100C002123331D002021161F5
:06127B0085820F0210C67F
:05128100050E0210C67D
:05128600150E0210C668
:07128B001204347800E2F5C3
:0A129200107A107BFF8A828B831212
:0B129C00187F7A117BFF8A828B83127F
:0512A700187F0210C6D3
:0712AC009043F712073E74A6
:0812B300FFC0E07443C0E074C9
:0812BB005FC0E07411C0E09077
:0C12C300F2BF12161DE58124FCF58174B9
:0812CF000BC0E07444C0E074A0
:0812D700EDC0E07410C0E090CE
:0C12DF00F33612161DE58124FCF5817425
:0812EB0017C0E07444C0E07478
:0812F30041C0E07411C0E0905D
:0C12FB00F24812161DE58124FCF581224A
:0E43E000303132333435363738396162636438
:0243EE00656602
:0743F00054454C454D20002F
:0243F7008B1227
:0643F90025440000000055
:0C43FF006D6F6E69746F725F70757400F2
:0C440B006D6F6E69746F725F67657400FE
:0E4417006D6F6E69746F725F626C696E6B0020
:0E4425006D203C30206F66662C2031206F6CBD
:0E443300642C203230207374643E0053657494
:0E44410020726164696F206D6F6E69746F7216
:04444F00696E67002B
:0A130700C01F85811FAA82AB83E09E
:0C131100FCA81F181818E6B5040E758221
:0C131D0003C002C003121411D003D00260
:07132900D21010AF02C21048
:0B1330008A828B83E060047C00800D4B
:0C133B008A828B83A81F181818E6F07C2B
:0113470001A4
:09134800A21092AF8C82D01F228A
:0A135100AA82AB83E0FC85158285BB
:0C135B001683A3A3A3A3A3E0FDECB5053B
:0E1367000E758203C002C003121411D003D011
:011375000275
:07137600D21010AF02C210FB
:0E137D008A828B83E060158A828B83C002C057
:07138B0003C022121841D03B
:0713920022D003D00280E429
:0A139900851582851683A3A3A3A384
:0C13A300A3E08A828B83F0A21092AF229C
:0A13AF00AA82AB83E0FC851582855D
:0C13B9001683A3A3A3A3A3E0FDECB505DD
:0313C50002800E95
:0E13C800758203C002C003121411D003D002BC
:0713D600D21010AF02C2109B
:0C13DD008A828B83E4F08A828B83C0221A
:0613E90012187FD022A2C1
:0413EF001092AF2287
:0613F300AA827B007C00D1
:0813F9008A051AED60118C0554
:071401001DEDFC60F38B04FC
:081408001CECFB60F40080F80D
:0114100022B9
:04141100AA82C2AF3A
:0C141500758214C0021213F3D0027B0594
:0E142100758201C002C0031221EE7582011215
:0C142F0013F37582011221F7758201127F
:0E143B0013F3D003D002DBDE758202C0021272
:0E14490013F3D002EA30E61C758201C00212D5
:0C14570021EE7582281213F37582011239
:0A14630021F775820A1213F3D0027C
:06146D00743F5AFB7C00F5
:0E147300C3EC9B509D758201C002C003C004F3
:0D1481001221EE75820A1213F3758201121A
:0E148E0021F775820A1213F3D004D003D002A6
:03149C000C80D4ED
:0344530071448031
:0344560079448026
:034459007E44801E
:03445C0082448017
:03445F008844800E
:034462008D448006
:03446500934480FD
:034468009A4480F3
:03446B009F4480EB
:03446E00A64480E1
:08447100737461727475700030
:0544790069646C6500A0
:04447E007061640005
:06448200626F6F7374000D
:05448800666173740081
:06448D00636F617374000F
:0744930064726F677565009C
:05449A006D61696E0078
:07449F006C616E64656400AE
:0844A600696E76616C69640027
:0C149F00AA82BA0A35780FE275F007A4A3
:0A14AB0024ADFBE434F3FC8B828CCB
:0E14B50083A3A3E0FBA3E0FCC002C003C004BD
:0A14C30074D3C0E07414C0E0C0034D
:0614CD00C00475820D222F
:0614D300D004D003D0029A
:0A14D900780FE275F007A424ADFBC4
:0C14E300E434F3FC8B828C83A3A3E0FBB9
:0C14EF00A3E0FCC003C0047405C0E0745E
:0A14FB0015C0E0C003C0048A82227D
:05150500D004D0032218
:0A150A00780FE275F007A424ADFA93
:0C151400E434F3FB8A828B83A3A3A3A31F
:0E152000E0FAA3E0FB4A600FC002C0038A821B
:09152E008B8312008BD003D00264
:011537002291
:06153800C2AF780FE2FAD9
:0B153E00EA75F007A424ADF582E43448
:0C154900F3F583E0FBA3E0FCC0028B8202
:0E1555008C8312008BAB82AC83D002BBFF1ED6
:0C156300BCFF1B0A7810E2B502027A00FF
:0C156F00780FE2B502C990F3BBC0021275
:06157B001841D00280BD02
:09158100780FEAF2D2AF8B82224E
:0A158A00780FE275F007A424ADFA13
:0C159400E434F3FB74062AF582E43BF516
:0515A00083E0F582224A
:0A15A500C01F85811FAA82AB837866
:0C15AF0010E2B4020E758207C002C003F7
:0715BB00121411D003D0024D
:0A15C2007810E275F007A4FC24ADD8
:0C15CC00F582E434F3F583EAF0A3EBF0C1
:0A15D800EC24ADFCE434F3FA8C823D
:0C15E2008A83A3A3E51F24FCF8E6F0A315
:0C15EE0008E6F08C828A83A3A3A3A3E587
:0C15FA001F24FAF8E6F0A308E6F07406DF
:0C1606002CF582E43AF5837401F07810B2
:0A161200E2FA781004F28A82D01F79
:01161C0022AB
:0A161D00C01F85811FAA82AB8374F1
:0C16270010B5140E758201C002C0031241
:061633001411D003D002E7
:021639007C0132
:05163B00EC60347D00AD
:0A164000C3ED95145023ED2D24BCDA
:0C164A00F582E434F3F583E0FEA3E0FF3A
:0E1656008E828F83A3A3A3A3A3E0FEB504029C
:02166400800301
:031666000D80D71D
:06166900EDB51402800340
:03166F000C80C923
:0E1672008A828B83A3A3A3A3A3ECF074062AA1
:0C168000F582E43BF583E51F24FAF8E650
:0E168C00F0A308E6F08A828B83E4F0A3F074EA
:0C169A00082AFCE43BFDE51F24FCF88658
:0E16A60006088607C002C0038E028C828D8368
:0E16B400EAF0A3AC82AD838F068C828D83EEAC
:0E16C200F0A3E4F0A37480F0A3AC82AD83D05B
:0516D00003D0027E0DB5
:0E16D5008C828D83E4F0A3AC82AD83DEF38AB9
:0C16E300828B83A3A3A3A37411F0D21088
:0516EF0010AF02C21063
:0516F400E5142514249B
:0A16F900BCF582E434F3F583EAF057
:0A170300A3EBF00514A21092AFD082
:02170D001F2299
:0E170F00C0E0C0A8C082C083C0F0C002C0030A
:0E171D00C004C005C006C007C000C001C0D097
:0A172B0075D000C01F74FFB517074A
:07173500E51414F517802CE8
:0A173C00E5812471FA8515828516F7
:0C17460083A3A3A3A3EAF074082515FBFD
:06175200E43516FC78905E
:0E1758008605088B828C83EDF0A3AB82AC83F8
:02176600DAF0B7
:0B17680075818FE5186004D2AF80028D
:02177300C2AF03
:02177500AA17B1
:051777000517E514B5A3
:05177C001703751700C2
:05178100E51725172407
:0A178600BCF582E434F3F583E0F5CE
:0617900015A3E0F516852B
:0A1796001582851683E0FBA3E0FC3A
:0817A000BB0005BC00028044FF
:0A17A800851582851683A3A3E0FBDC
:0E17B200A3E0FC4B6022C002122E3AAB82ACC8
:0A17C00083D002851582851683A3ED
:0E17CA00A3E0FDA3E0FEEBC39DFBEC9EFC3014
:0217D800E71216
:0A17DA00EAB51799E5187095D2AF33
:0817E400758701C2AF021777FF
:0A17EC00851582851683A3A3A3A32D
:0C17F600E0FA748F2AF58174082515FBB9
:06180200E43516FC7890AD
:0E1808008B828C83E0FDA3AB82AC83A6050827
:0C181600DAF0D01FD0D0D001D000D007F5
:0E182200D006D005D004D003D002D0F0D08381
:0C183000D082D0E020E705C2AF02183ED5
:02183C00D2AF29
:03183E00D0E022D5
:0A184100AA82AB8385158285168309
:0C184B00EAF0A3EBF012170F8515828560
:0B1857001683E0FAA3E0FB4A601A854C
:0A1862001582851683E4F0A3F085DB
:0A186C001582851683A3A3E4F0A300
:05187600F07582012263
:04187B007582002250
:06187F00AA82AB837C008D
:0A188500C3EC9514502CEC2C24BC8D
:0C188F00F582E434F3F583E0FDA3E0FEF5
:0E189B008D828E83E0FFA3E0F8EFB5020CE82B
:0B18A900B503088D828E83E4F0A3F0ED
:0318B4000C80CED7
:0118B700220E
:0B18B800AA82AB8374022515FCE43506
:0B18C30016FDC002C003C004C00512E7
:0E18CE002E3AE5828583F0D005D004D003D0F9
:0C18DC00022AFAEB35F0FB0ABA00010BFF
:0E18E8008C828D83EAF0A3EBF0EA4B700E8544
:0A18F6001582851683A3A37401F088
:03190000A3E4F06D
:0119030022C1
:0A190400851582851683A3A3E4F085
:03190E00A3F02221
:071911001218B890F3DC127C
:05191800184102190452
:07191D00C2AF1514AA1775F3
:0219240017FFAB
:0A192600C3EA95145029EA2A24BCF4
:0B193000FBE434F3FCEA04FD25E02496
:0A193B00BCF582E434F3F583E0FE0E
:0E194500A3E0FF8B828C83EEF0A3EFF08D0207
:0219530080D141
:06195500E4F515F5160291
:02195B00170F64
:02195D007A000E
:0A195F00C3EA9514504FEA2A24BC95
:0C196900F582E434F3F583E0FBA3E0FC1E
:0E1975008B828C83E0FDA3E0FE74062BF582CE
:0E198300E43CF583E0FBA3E0FC7F80C002C0E3
:0C19910005C006C003C004C00774AEC04F
:0C199D00E07444C0E07480C0E0123A70B6
:0B19A900E58124F8F581D0020A80AB34
:0119B4002210
:0719B5007517FFE4F515F5BD
:0419BC001602170FE9
:0E44AE00253132733A20776368616E20253025
:0444BC0034780A0046
:0A19C000C01F85811FC082C083C0D4
:0C19CA00F0C0E07811E4F208F208F20826
:0A19D600F27815E4F278167445F279
:0D19E0000874AFF20874FCF20874FFF2A85E
:0C19ED001F08E6248AFE08E6345EFF08AE
:0C19F900E634F9FA08E634FFFBA81F08EA
:0E1A0500A60608A60708A60208A603EB30E70F
:0A1A13001878157401F2A81F08C32B
:0E1A1D00E496F608E496F608E496F608E496D9
:011A2B00F6C4
:0C1A2C00A81F088602088603088604082C
:021A3800860521
:0C1A3A007816C3E2F5F0E495F008E2F540
:0E1A4600F0E495F008E2F5F0E495F008E2F522
:0C1A5400F0748063F08095F0502C781640
:0E1A6000E2248AF208E2345EF208E234F9F27F
:0C1A6E0008E234FFF27811E22401F208D3
:0E1A7A00E23400F208E23400F208E23400F236
:021A880080B02C
:0A1A8A007816E51F24FAF9E227F2AE
:0E1A940008E20937F208E20937F208E20937E2
:0E1AA200F21ABAFF091BBBFF051CBCFF011D99
:071AB000ED20E703021A3AE2
:0A1AB7007815E2601A7811E2D3F40A
:0E1AC1003400F208E2F43400F208E2F43400DB
:071ACF00F208E2F43400F21A
:0A1AD600E51F24FAF87911E326FA5F
:0E1AE00009E30836FB09E30836FC09E3083683
:0A1AEE008A828B838CF0851F81D063
:021AF8001F22AB
:0A1AFA00C01F85811FE582FAF4FB8E
:0C1B0400E5905203A81F181818E65202C2
:091B1000EA4BF5900000D01F2201
:0A1B1900AA8243902043FE207B08BF
:081B23007C00EA30E7027C209F
:0E1B2B00EA2AFA74104CFDC002C003C004C0C8
:0D1B390005758230121AFA1581758230127E
:0E1B46001AFA1581D003D002DBD353FEDF2242
:041B54007A007B0890
:0E1B5800EA2AFAC002C0037410C0E0758210C1
:0E1B6600121AFA1581D003D002309503430203
:011B7400016F
:0E1B7500C002C003E4C0E0758210121AFA1517
:0A1B830081D003D002DBCE8A82225B
:0E1B8D00AA82758255C002121B19D0028A82EC
:061B9B00121B19021B548D
:0A1BA100C01F85811FAA82758256BD
:0D1BAB00C002121B19D0028A82121B19A859
:0A1BB8001F1818188682121B19125C
:051BC2001B54D01F229E
:0A1BC700C01F85811FAA8275825796
:0D1BD100C002121B19D0028A82121B19A833
:0A1BDE001F1818188682121B19E563
:0A1BE8001F24FCF88682121B19125C
:051BF2001B54D01F226E
:0E1BF700AA82AB83758200C002C003121B8D50
:0C1C0500E582781AF274D0C0E07582E528
:0C1C1100121BA1AC821581781BECF27450
:0E1C1D0082C0E07582E5121BA1AC82158178B1
:0B1C2B001CECF27483C0E07582E5122F
:0C1C36001BA1AC821581781DECF27484B7
:0D1C4200C0E07582E5121BA1AC821581780F
:0B1C4F001EECF27485C0E07582E51207
:0C1C5A001BA1AC821581D003D002781FC2
:0E1C6600ECF28A048B02C004C0027582901258
:071C74001BC7158115812239
:0C1C7B00781CE2C0E07482C0E075827545
:0C1C8700121BC715811581781DE2C0E01A
:0E1C93007483C0E0758275121BC71581158120
:0C1CA100781EE2C0E07484C0E07582751B
:0C1CAD00121BC715811581781FE2C0E0F2
:0E1CB9007485C0E0758275121BC715811581F8
:0C1CC700781BE2C0E074D0C0E0758275AC
:0C1CD300121BC715811581781AE2C0E0D1
:091CDF00758274121BA11581220B
:0E1CE800AA82C002758274121BA1158175823A
:0A1CF600F0121B8D7582A3021B8DF6
:0C1D00007582E0121B8D7582A3021B8D02
:0E1D0C0053F4C743F62043901843FE1853FECD
:021D1A00DF22C6
:021D1C007A1437
:041D1E0000DAFD22C8
:0C1D2200AA82C002121D1CD002C0198A47
:071D2E0082121AFA1581224E
:0C1D3500AA82C002121D0C7519387582BC
:0C1D410038121D22D00274204AFB8B19BE
:0E1D4D00758238C002C003121D2290000A12D7
:0E1D5B0019117430C0E0758238121AFA158121
:0B1D6900D0038B19758238121D227503
:0C1D74001930758238121D22D00274282C
:0C1D80004AF519758238121D2290000AE5
:031D8C0002191128
:061D8F00758200021D3503
:061D9500758210021D35ED
:0A1D9B0012037E7806E2B40A01226A
:091DA5001204347807E2700A7898
:091DAE0000E2F582121B1980E429
:011DB7002209
:091DB8001204347807E2600122F4
:0C1DC1007800E2FA08E2FBC3E49A740127
:091DCD009B500678077402F22213
:041DD6007C007D0010
:0E1DDA00C3EC9AED9B5042EC4D601BEC54079D
:0E1DE800701675820AC002C003C004C0051246
:0A1DF600149FD005D004D003D002E2
:0E1E0000C002C003C004C005121B5412034AE6
:0E1E0E0075822012149FD005D004D003D0029C
:071E1C000CBC00BA0D80B7F9
:061E230075820A02149F03
:0C1E29001204347800E2FA08E2FBC00268
:0C1E3500C003120434D003D0027800E295
:0A1E4100FC08E2FD7807E2600122D0
:0E1E4B008C828D83C002C003121BF7D003D01F
:031E5900027C0008
:091E5C008A058B061ABAFF011B6E
:0E1E6500ED4E602E8C050CED54077012758248
:0E1E73000AC002C003C00412149FD004D003A2
:021E8100D0028D
:0E1E8300C002C003C004121D0012034AD004A6
:061E9100D003D00280C561
:091E9700121C7B75820A02149FE3
:0C1EA0001204347800E2FA08E2FBC002F1
:0C1EAC00C003120434D003D0027800E21E
:0A1EB800FC08E2FD7807E260012259
:0E1EC2008C828D83C002C003121BF7D003D0A8
:011ED000020F
:091ED1008A048B051ABAFF011BFB
:0E1EDA00EC4D6032C002C0031202DBE582C490
:0E1EE80054F0FCC0041202DBAD82D004D00323
:0B1EF600D002ED42047807E2600122F8
:0E1F01008C82C002C003121CE8D003D0028004
:011F0F00C110
:031F1000021C7B35
:061F13009044C002073EED
:0244C0008F1D4E
:0244C200DC44D8
:0244C400B81D21
:0244C600EB44C5
:0244C800291EAB
:0244CA00FE44AE
:0244CC00A01E30
:0244CE00274580
:0244D0009B1D32
:0244D200514552
:0244D400951D34
:0644D60067450000000034
:0E44DC004400456E61626C6520646562756720
:0144EA0000D1
:0E44EB0047203C636F756E743E004765742079
:0544F900646174610024
:0E44FE0049203C636F756E743E203C6164641F
:0E450C00723E00496E707574203C636F756ED0
:0D451A00743E206174203C616464723E00B8
:0E4527004F203C636F756E743E203C616464EF
:0E453500723E004F7574707574203C636F7594
:0E4543006E743E206174203C616464723E0020
:0E45510050203C627974653E202E2E2E0050C4
:08455F007574206461746100B1
:084567005200526573657400F7
:041F190075B6B022C7
:0A1F1D00E51A14541F25E025E02406
:051F2700DDF54FE4347C
:041F2C00F3F5507504
:061F30005104E4F5520229
:021F36002D9FDD
:0C1F3800C022C0E0C0F0C082C083C00224
:0E1F4400C003C004C005C006C007C000C00135
:0C1F5200C0D075D000E5B5E51A25E025EB
:0A1F5E00E024DDFAE434F3FB740222
:0E1F68002AFAE43BFB8A828B83E5BAF08A8278
:0C1F76008B83A3E5BBF0E51A25E025E015
:0A1F820024DDFAE434F3FBC002C0D2
:0E1F8C0003122E3AAC82AD83D003D0028A82BB
:0C1F9A008B83ECF0A3EDF0E51A04541F5B
:0A1FA600F51A7A1A7BFF8A828B83FA
:0E1FB00012187FD0D0D001D000D007D006D0BC
:0E1FBE0005D004D003D002D083D082D0F0D062
:041FCC00E0D022320D
:071FD00090F45D121F1D904B
:0E1FD700F45FE0FAA3E0FB90F45DE0FCA3E011
:0C1FE500FDC002C003C004C005746FC042
:0C1FF100E07445C0E07480C0E0123A705B
:071FFD00E58124F9F58122C2
:0E20040075F201C28D43A80290458302073E8B
:0E456F007469636B3A2025357520626174749F
:06457D00202535640A0050
:02458300D01F47
:064585008B450000000060
:0E458B00610043757272656E742041444300F6
:0C201200AA82AB837405B5230E75820210
:0B201E00C002C003121411D003D00256
:08202900AC230523EC2CFD247F
:0A20310089F582E434F4F583EAF047
:0E203B00A3EBF0EC701FF5D1C2C043B8017AE0
:06204900617BF48BD57AE7
:06204F00617BF48AD47AE3
:06205500697BF48BD37AD5
:05205B00697BF48AD24C
:032060008C82224D
:0C206300AA828AF005F07B017C00800658
:06206F00EB2BFBEC33FC3F
:0E207500D5F0F7ADD67E00ED5203EE5204EB2F
:0D2083004C600A758202C002121411D002D6
:0C209000EAC40354F8FA2461F582E43439
:06209C00F4F583AB24AC57
:0A20A200258C05EDF0EA2461FAE454
:0C20AC0034F4FD8A828D83A3EBF08A825D
:0A20B8008D83A3A3AB26AC278C0692
:0E20C200EEF08A828D83A3A3A3EBF08A828DB9
:0C20D00083A3A3A3A3E529F08A828D83DB
:0C20DC00A3A3A3A3A3E528F074062AF533
:0C20E80082E43DF583E52AF074072AF538
:0B20F40082E43DF5837408452BF022C8
:0A20FF00AA828AF005F07401800245
:0221090025E0CF
:0E210B00D5F0FBFBF4FC52D1EB55D6600D7401
:0C211900804BF5D6000000000000000024
:0A212500EA2A2489F582E434F4F577
:0E212F0083E0FAA3E0FC8A828C83E4F08BD676
:0A213D000000000000000000002276
:0A214700AA828AF005F074018002FC
:0221510025E087
:06215300D5F0FB42D7228B
:0A215900AA828AF005F074018002EA
:0221630025E075
:0E216500D5F0FBFA74804AF5D6EAF452D12286
:0C217300C022C0E0C0F0C082C083C002E7
:0E217F00C003C004C005C006C007C000C001F8
:0B218D00C0D075D0007A017B007C0000
:0C219800C3EC95235033EA55D16026C2F9
:0C21A400C0EAF4F5D1EB2B2489F582E4AD
:0C21B00034F4F583E0FDA3E0FE8D828E88
:0D21BC00837401F08D828E8312187F8008DD
:0821C900EA2AFA0C8C0380C71E
:0E21D100D0D0D001D000D007D006D005D00469
:0D21DF00D003D002D083D082D0F0D0E0D069
:0221EC0022329D
:0921EE00AA827820E25A429022F4
:0C21F700AA827820E25202EAF452902200
:0C220300AA827820E2F4FBE590520378F8
:07220F0020E25A4BF590227A
:09221600AA827820E25A629022AB
:0A221F00C01F85811FAA82C00212B1
:0C22290021EEE51F24FCF8868208868365
:0B223500121911D0028A821221F7D08A
:022240001F225B
:0C224200AA827820EAF2EAF4FB52F4EBE6
:06224E005290EA42FE225C
:0C2254007582011221EE7823E2603690C2
:07226000F4E2E07030754F5D
:032267002D755082
:05226A00F57823E2F508
:05226F005175520090C2
:06227400F4E5122D9F901D
:07227A00F4E27823E2F0908A
:0B228100F4E3E0FA0A90F4E3EAF078DE
:07228C0023E4F290F52D128E
:02229300187FB2
:0E229500744CC0E090F4E112276B1581758245
:0422A300010221F71C
:0E22A700E4C0E0744EC0E090F4931227E2AA67
:0B22B5008215811581EA7003F582227A
:0C22C00090F4E0E0FA20E70475820022B0
:0822CC00740724F3F54FE4341C
:0422D400F0F550755C
:0622D8005108E4F55290EC
:0A22DE00F4D7122DF8E582601C7A97
:0422E800997B458A0F
:0422EC004F8B50754F
:0622F0005107E4F55290D5
:0D22F600F0FA122DF8E582600475820022D6
:0E23030090F494E0FABAFF1890F495E0FB789D
:0823110024F290F496E0FC9028
:0A231900F4E3F090F4E4EBF0805AD6
:0C232300EA605790F495E0FB7824E22477
:08232F0001FCEBB5040280077C
:0723370090F625E0FB603F7A
:0A233E0078227921E2F5F0E3B5F012
:092348003474042493F54FE434CD
:04235100F4F5508AC5
:052355005175520090DB
:06235A00F56D122D9F78C5
:0823600022E4F290F494E0780D
:0823680021F290F495E0FA78EF
:0823700024F290F4E4EAF0907D
:05237800F3BB12187F09
:0B237D0090F625E4F090F496E0FA9052
:0E238800F4E3E0FBEAB5030B90F4E2E4F0901E
:05239600F4E112187FC4
:04239B007582012224
:0C239F007823E2600D90F626E0FA60065C
:0623AB0090F62602187FE7
:0123B1002209
:0223B200AA82FD
:0C23B4007823E2B4401690F624E0FB60B1
:0A23C0000FC00212239F90F52D12AA
:0623CA001841D00280E47E
:0C23D00090F624E0FB60147823E2FB7818
:0A23DC002304F2EB242DF582E43413
:0523E600F5F583EAF0AB
:0123EB0022CF
:0B23EC0090F624E0FA700490FFFF223E
:0A23F70078227921E2F5F0E3B5F059
:052401000490FFFF2222
:0A2406007822E2FA782204F2EA24B8
:0A2410006DF582E434F5F583E0FA7F
:07241A007B008A828B832204
:074599004E3043414C4C0081
:0E2421001223ECAA82AB838A048B05BAFF2239
:0E242F00BBFF1F90F624E0FA601890F626E03E
:09243D00FA600690F62612187FE1
:0724460012150A90F3BB120E
:04244D00184180D0E2
:052451008C828D832246
:0E24560090F624E0FA6016122421AA82AB83CD
:08246400BAFF05BBFF0280EA8C
:07246C008A8212149F80E335
:0324730002191D2E
:0E24760090F69E740AF0E4A3F0122E3AE5826E
:0C2484008583F090F6A0F0A3E5F0F022B4
:0E24900090F69EE0FAA3E0FBBA0A31BB002EE4
:0E249E00122E3AAA82AB8390F6A0E0FCA3E0D7
:0E24AC00FDEAC39CFAEB9DFBC374C89A7480D2
:0E24BA008BF063F08095F0500990F69E7464EC
:0424C800F0E4A3F0A9
:0124CC0022ED
:0D24CD00120A069000A4E493FA74019390A3
:0B24DA00F4E1EAF090F4E274FFF0126D
:0E24E5002E3AE5828583F090F6A0F0A3E5F094
:0A24F300F090F69E740AF0E4A3F0E6
:0A24FD0090F624E0FA700302259C1B
:08250700740724F3F54FE434DE
:04250F00F0F550751E
:062513005108E4F55290AE
:06251900F525122D9F12B2
:09251F00225490F4E2E060031282
:02252800247617
:0E252A0012249090F12DE0FAE4CA25E0CA33A5
:0A253800FB8AF005F090000A800B0A
:0B254200E5822582F582E58333F583F6
:0E254D00D5F0F21218B81222A7AA82C002120C
:0C255B001904D002EA609B7823E26006BD
:0625670090F4E2E0609038
:09256D0090F494E060031224765E
:0E25760090F6267401F090F69EE0FAA3E0FBCA
:0B2584008A828B831218B890F6261292
:06258F001841121904902E
:07259500F626E4F00224FD2C
:03259C0002191D04
:0A259F0090F6247401F012037E127E
:0625A900150A12128174F4
:0825AF00A0C0E07445C0E07417
:0825B700CDC0E07424C0E090E7
:0C25BF00F5AD12161DE58124FCF58174B9
:0825CB00A7C0E07445C0E074F4
:0825D30056C0E07424C0E09042
:0B25DB00F62712161DE58124FCF58197
:0C25E600121538AA828A03BA7E02800C0B
:0525F200BB0D027B0A95
:0725F7008B821223B280E881
:0225FE007A0061
:0B2600007823E2700690F4E2E0601521
:0E260B00C3EA6480948A500D90000AC0021247
:072619001911D0020A80E054
:0526200090F624E4F037
:0E26250090F627E0FAA3E0FB4A700B90F5ADAB
:08263300E0FAA3E0FB4A60118C
:07263B001228F190F3BB121D
:0A264200187F90000112191180D9D1
:03264C00021286F1
:0E264F0090F6A7E0FA3395E0FBC002C00374DA
:0A265D00ACC0E07445C0E07480C01A
:0B266700E0123A70E58124FBF58122AF
:062672009045B602073E90
:0745A0006D61737465720088
:0545A7006563686F0070
:0A45AC00525353493A2025640A00D7
:0245B6009F253F
:0245B800C245FA
:0245BA004F268A
:0645BC00D84500000000DC
:0E45C200700052656D6F7465207061636B65EB
:0845D00074206C696E6B2E0073
:0E45D80073005265706F7274207369676E61B4
:0C45E6006C20737472656E6774682E00A0
:0C267800C022C0E0C0F0C082C083C002DD
:0E268400C003C004C005C006C007C000C001EE
:0E269200C0D075D000539BFCE5E930E508127E
:0726A00028F153E9DF80146B
:0E26A700E5E930E40F90F6A47401F090F6A47B
:0626B50012187F53E9EF4B
:0E26BB00D0D0D001D000D007D006D005D0047A
:0D26C900D003D002D083D082D0F0D0E0D07A
:0226D6002232AE
:0226D8007A0086
:0326DA00BA0A0039
:0D26DD005018EA90465093FB7CDFEA049011
:0D26EA00465093FD8B828C83F00A0A80E33A
:0126F70022C0
:0926F80090DF3BE0FABA01012277
:0E27010075E10412170F90DF3BE0FABA01F207
:01270F0022A7
:0B271000AA82C002120A0690F6A61270
:0D271B0013511226F8D00290DF06E4F09072
:0D272800F110E0FBA3E0FCA3E0FDA3E090B6
:0E273500DF09EDF090DF0AECF090DF0BEBF027
:0D27430090DF02EAF090F12DE025E0FA9021
:0C275000465A9390DF0CF0EA245AFAE499
:0B275C003446FB8A828B83A3E4939039
:04276700DF11F0226C
:0A276B00C01F85811FAA82AB83A85E
:0B2775001F1818188682C002C0031253
:0C2780002710D003D00290F6A4E4F090E3
:0A278C00F6A2E0FCA81F181818863A
:05279600287529008AEE
:04279B00248B2575F1
:06279F0026D97527DF7545
:0827A5002A13752B428C8212ED
:0927AD00206390F6A2E0F582120F
:0B27B60020FF75E103D21010AF02C23B
:0127C1001007
:0B27C20090F6A4E0FA700C90F6A4C0A2
:0527CD0022121841D0AA
:0327D2002280ED75
:0827D500A21092AF90F6A612CB
:0527DD0013AFD01F2224
:0A27E200C01F85811FAA82AB8390FF
:0C27EC00F6A5E4F0A81F181818E624FE5B
:0E27F800F582C002C003122710D003D0029059
:0A280600F6A2E0FCA81F18181886BF
:05281000287529007588
:0628150024D97525DF8ABD
:04281B00268B27756C
:0A281F002A13752B128C82C002C030
:0B2829000312206390F6A2E0F582127B
:0C28340020FFD003D00275E102E51F2454
:0C284000FCF8E66018E51F24FCF8860494
:0E284C007D008C828D83C002C0031218B8D0AC
:03285A0003D002A6
:07285D00D21010AF02C210FF
:0E28640090F6A3E0FC701D90F6A5E0FC701647
:0A28720090F6A3C002C003C02212BA
:0C287C001841E582D022D003D00260DCBD
:0A288800A21092AFE51F24FCF8E651
:0D289200600BC002C003121904D003D00275
:0E289F0090F6A3E0FC701390F6A2E0F5821212
:0628AD0021591226F890EB
:0628B300F6A7E4F0802905
:0C28B900A81F18181886047D00EC24FEEF
:0E28C500FCED34FFFDEC2AF582ED3BF583E0DF
:0E28D300A2E713FA3395E0FBEA24B690F6A7CD
:0128E100F006
:0728E20090F6A61213AF905F
:0828E900F6A3E0F582D01F22E6
:0A28F10090F6A57401F090F6A30222
:0228FB00187F44
:0C28FD0090F6A5E4F075827D1227109083
:06290900F6A4E4F07A00E0
:03290F00BA0E00FD
:0D2912005018EA90464293FB7CDFEA0490E7
:0D291F00464293FD8B828C83F00A0A80E310
:01292C002288
:0D292D0090F6A2E0F5821220FF75E103D2C2
:06293A000010AF02C20014
:0E29400090F6A4E0FA700F90F6A5E0FA700889
:08294E0090F6A412184180EA82
:0C295600A20092AF90F6A4E0FA700C9082
:09296200F6A2E0F58212215912DF
:02296B0026F84C
:07296D001226D890F6A60225
:0229740013AF9F
:092976001228FD90F6A2E0FA7BA4
:04297F00607C468BA7
:04298300248C257506
:0629870026D97527DF755B
:06298D00287DE4F5297528
:082993002A13752B028A82123F
:05299B00206302292D5C
:0E29A000AA82C0021228FDD00290F6A2E0FB2F
:0C29AE007403C39AC42354E02462FAE4CA
:0629BA003446FC8A248C67
:0529C000257526D97504
:0729C50027DF752878E4F517
:0529CC0029752A1375B6
:0829D1002B428B8212206302ED
:0229D900292DA6
:0A29DB0090F6A57401F090F6A40236
:0229E500187F59
:0E29E700E582FA602190F6A8E0FAA3E0FB4A30
:0E29F50070341212817582FF12271075E103F3
:0A2A030090F6A87401F0E4A3F0229D
:0E2A0D0090F6A8E0FAA3E0FB4A60131226F848
:072A1B0090F6A61213AF9024
:092A2200F6A8E4F0A3F00212860C
:012A2B002288
:0C2A2C007A02C00212037ED0027806E29B
:052A3800B40A02800752
:072A3D0012048D7802E2FA99
:0E2A44000AEA30E10A758201C0021229E7D0C9
:012A52000281
:0A2A5300BA0325C002741AC0E07433
:0C2A5D0047C0E07480C0E0123A701581A0
:0E2A69001581158112150A12153875820A1290
:042A7700149FD002D6
:0A2A7B00EA30E0067582000229E748
:012A8500222E
:082A86001204347800E2FA7832
:052A8E0007E2600122D7
:0E2A9300C002120434D0028A827583DFE0FB99
:0E2AA1007C008A057E00C002C003C004C00590
:0A2AAF00C0067435C0E07447C0E0B3
:0E2AB9007480C0E0123A70E58124F9F581D0F6
:0C2AC700027807E2702B8A827583DF78AA
:0C2AD30000E2F08A827583DFE0FA7B00ED
:0A2ADF00C002C003743FC0E074475A
:0E2AE900C0E07480C0E0123A70E58124FBF575
:012AF700815D
:092AF8007807E4F27446C0E074B2
:0C2B010047C0E07480C0E0123A701581FB
:052B0D00158115812275
:022B12007A0047
:032B1400BA5000B4
:0D2B17005018EA9045F293FB7CDFEA049031
:0D2B240045F293FD8B828C83F00A0A80E35A
:0A2B31001226D890F6A37401F012EA
:0E2B3B002012E58290F6A2F075E90075913047
:092B4900439A0190474802073E3F
:0E45F20027C028C029C02AC02BC02CC02DC055
:0E4600002EC0070608000DA30E110FA2101108
:0E460E0006001B101A561CE91D0A1E001F1F75
:0E461C0023812435250900D301910324044491
:0E462A00050012071330141815001660170350
:0A463800180019002F0030003100B7
:0E4642000CD60D5E0E900F0211160300040040
:0A4650000DA30E110FA20324044471
:06465A00DA36F816F60046
:02466000550003
:0E46620000000000000000000000000000004A
:0E4670000000000000000000000055555555E8
:0E467E005555555500000000000000000000DA
:0E468C00000000000000000000000000000020
:0E469A0055555555555555550000000000006A
:0E46A800000000000000000000000000000004
:0E46B60000000000555555555555555500004E
:0E46C4000000000000000000000000000000E8
:0E46D2000000000000000000000000000000DA
:0E46E0000000000000000000000000000000CC
:0E46EE000000000000000000000000000000BE
:0E46FC000000000000000000000000000000B0
:0E470A000000000000000000000000000000A1
:0247180000009F
:0E471A00486974206120636861726163746590
:0D4728007220746F2073746F702E2E2E009F
:0A47350052465B25785D20257800D0
:07473F00202D3E202578002B
:024746000A0067
:024748002C2A19
:02474A005447D2
:02474C00862ABB
:06474E0086470000000098
:0E47540043203C312073746172742C2030209D
:0E47620073746F702C206E6F6E6520626F7422
:0E477000683E00526164696F20636172726975
:08477E0065722074657374007C
:0E47860056203C6F66667365743E203C76617B
:0E4794006C75653E0053657420726164696F38
:0A47A2002072656769737465720088
:0200A00002005C
:0200A200FDFF60
:0200A40000005A
:0400A600331B1200F6
:0C2B5200C022C0E0C0F0C082C083C002FE
:0E2B5E00C003C004C005C006C007C000C0010F
:0E2B6C00C0D075D00090F6ACE0FA7B000ABA3B
:032B7A0000010B4C
:0E2B7D0053021F7B0090F6ADE0FC7D00EAB530
:082B8B000406EBB50502801CF5
:0A2B930090F6ACE024AEF582E434C5
:0C2B9D00F6F583E5F9F090F6ACE0045486
:062BA9001FFA90F6ACF0EB
:072BAF0090F6AC12187F90B4
:0E2BB600F3BB12187FD0D0D001D000D007D0D2
:0E2BC40006D005D004D003D002D083D082D03A
:062BD200F0D0E0D0223239
:0E2BD80090F6CEE0FA90F6CFE0FBEAB50301EE
:012BE60022CC
:0E2BE70090F6F0E0FA702290F6F07401F09093
:092BF500F6CFE024D0F582E434AF
:0C2BFE00F6F583E0F5F990F6CFE0045402
:062C0A001FFA90F6CFF066
:012C100022A1
:0C2C1100C022C0E0C0F0C082C083C0023E
:0E2C1D00C003C004C005C006C007C000C0014F
:0D2C2B00C0D075D000C2EA90F6F0E4F012BF
:062C38002BD890F6CE122D
:0E2C3E00187FD0D0D001D000D007D006D0052E
:0E2C4C00D004D003D002D083D082D0F0D0E0EC
:032C5A00D0223253
:052C5D00D310AF01C31C
:022C6200C0D0E0
:0E2C640090F6ACE0FA90F6ADE0FBEAB503089E
:082C720090F6AC12184180EA53
:0A2C7A0090F6ADE024AEF582E434DC
:0C2C8400F6F583E0FA90F6ADE004541F72
:0B2C900090F6ADF08A82D0D092AF2207
:0E2C9B0090F6ACE0FA90F6ADE0FBEAB503046B
:042CA90090FFFF2277
:0A2CAD0090F6ADE024AEF582E434A9
:0C2CB700F6F583E0FA90F6ADE004541F3F
:0B2CC30090F6ADF07B008A828B83222C
:052CCE00D310AF01C3AB
:042CD300C0D0AA8241
:0C2CD70090F6CEE0FB7C000BBB00010C73
:0E2CE30053031F7C0090F6CFE0FD7E00EBB5A2
:0E2CF1000510ECB5060C90F6CEC0021218418C
:042CFF00D00280D4AB
:0A2D030090F6CEE024D0F582E4340F
:0C2D0D00F6F583EAF090F6CEE004541FC7
:0C2D190090F6CEF0122BD8D0D092AF2252
:052D2500D310AF01C353
:022D2A00C0D017
:0E2D2C0090F6CEE0FA90F6CFE0FBEAB5030297
:022D3A0080080F
:082D3C0090F6CE12184180E868
:052D4400D0D092AF2287
:0E2D4900AA82C002122D25D002EA24FB5001FE
:012D57002259
:0E2D580043FB80EA2AFA9047AC93F5FAEA248E
:0A2D6600ACFAE43447FB8A828B8349
:062D7000A3E493F5FC2230
:0E2D760053F1FDAAFF743F5AF5F0744045F08A
:0E2D8400F5FF43F33043F30C75F8C075820081
:0D2D9200122D4975FBC243A808439A082280
:0A47AC00A307A308A3093B0B3B0C75
:082D9F00AA82AB83AC51AD52D6
:092DA7008C068D071CBCFF011D08
:0A2DB000EE4F601FAE4FAF508E8251
:0E2DBA008F83E0F88A828B83F00ABA00010B47
:0A2DC80074012EF54FE43FF5508032
:012DD200D42C
:012DD30022DD
:082DD400AA82AB83AC50AD51A3
:092DDC008C068D071CBCFF011DD3
:0C2DE500EE4F600E8A828B83E54FF00AEF
:062DF100BA00E80B80E5CA
:012DF70022B9
:082DF800AA82AB83AC51AD527D
:092E00008C068D071CBCFF011DAE
:0C2E0900EE4F60298A828B83E0FEAF4F01
:0C2E1500A8508F828883E0F9EEC399FE7C
:052E210060038E822217
:052E26000ABA00010BD7
:0A2E2B0074012FF54FE438F55080D4
:012E3500CAD2
:042E3600758200227F
:0301A600751D01C3
:052E3A00D310AF01C33D
:0A2E3F00C0D0851B82851C83D0D013
:032E490092AF2223
:0C2E4C00C022C0E0C0F0C082C083C00201
:0E2E5800C003C004C005C006C007C000C00112
:0A2E6600C0D075D0007401251BF5E3
:052E70001BE4351CF518
:042E75001C051EE535
:052E79001DB51E0675E9
:052E7E001E00121F19E7
:0E2E8300D0D0D001D000D007D006D005D004AA
:0D2E9100D003D002D083D082D0F0D0E0D0AA
:022E9E002232DE
:052EA000D310AF01C3D7
:0A2EA500C0D085821D751E00D0D03C
:032EAF0092AF22BD
:0E2EB20075E40075DB7575DA3075E50475E6BC
:0E2EC0000075E70075E200D2DED2B975E406B7
:012ECE0022E1
:042ECF007A007B000A
:052ED3001ABAFF011B0B
:072ED800EA4B60030080F4E7
:012EDF0022D0
:0E2EE00053BEFBAAC674BF5AF5F0744045F00D
:022EEE00F5C627
:0B2EF000E5BE30E5FB122ECF53C6BF3D
:0B2EFB00E5BE30E6FB43BE0453C6C03A
:082F0600E5C6543F600280F8AB
:012F0E0022A0
:0D2F0F0090DE077421F090DE097410F09040
:062F1C00DE0B7404F0223C
:0C2F2200C022C0E0C0F0C082C083C0022A
:0E2F2E00C003C004C005C006C007C000C0013B
:0D2F3C00C0D075D000C2E890DE02E0FA7847
:0A2F490027E24AF27827E254016003
:072F53000690F6F112187F51
:0B2F5A007827E25420600690F7681210
:022F6500187FD3
:0E2F670090DE04E0FA30E40690F3BB12187F0F
:0B2F750090DE06E0FA30E203122F0F9E
:0E2F8000D0D0D001D000D007D006D005D004AC
:0D2F8E00D003D002D083D082D0F0D0E0D0AC
:022F9B002232E0
:0E2F9D0090DE0EE4F090DE11E0FA30E1012249
:0A2FAB00782DE2FB24DF50027B20AA
:072FB5007A02BB2002800636
:062FBC007A0A7829E4F214
:062FC200782DE2C39BF232
:0C2FC8008B041BEC6028782AE2FC08E275
:0E2FD400FD08E2FE8C828D838EF0124036FFE7
:0C2FE200782A74012CF2E43D08F208EE9D
:082FEE00F290DE20EFF080D22A
:0B2FF60090DE0EE4F090DE11EAF02205
:08300100AA82AC837BAA7D00CA
:0E3009008B828D83E493FE60408B828D83A3C7
:0E301700E493FFB504278A071AEF7021BC026C
:0C3025000E8B828D83A3A3E493FF782D13
:03303100F2800426
:04303400782DEEF213
:0C303800782AEBF208EDF2087480F22216
:0E3044008B828D83E493FE2BFBE43DFD80B771
:01305200225B
:0C30530090DE0EE4F090DE16E0FA78301B
:09305F00C3E29A50047830E2FA51
:063068007830E2C39AF289
:0C306E008A031AEB601D7831E2FB08E2D7
:0C307A00FC90DE20E0FD8B828C83F0785F
:0B3086003174012BF2E43C08F280DD05
:01309100221C
:0A309200AA82782DE2FB782D04F2EB
:07309C00EB242EF8EAF222FA
:0C30A300AA8278287401F290DE00EAF0A6
:0130AF0022FE
:0D30B00090DE0E7405F090DE107408F090B4
:0D30BD00DE12E04401F090DE0E7404F0908D
:0C30CA00DE137408F090DE157401F02293
:0730D6007831746CF20874FC
:0830DD00F7F278307408F212DA
:0830E50030537830E260012253
:0A30ED00782A742EF208E4F2087449
:0C30F70060F2782DE4F290F76CE0FA74BF
:0B310300605AFB6009BB20030231CBC7
:03310E000231FB90
:0831110053021FBA0002800FF7
:06311900BA01030231922D
:06311F00BA02030231B404
:033125000231FB79
:0C31280090F76DE0FA6017BA05028021F4
:05313400BA0602802B29
:05313900BA0802803815
:05313E00BA0902803E09
:033143000231FB5B
:0D31460075820012309275820012309202E4
:0231530031FB4E
:0D31550090F76EE0FAA3E08A821230A30228
:0231620031FB3F
:0D31640090F76EE0FAA3E0FB8A828B8312E5
:0531710030010231FBFA
:093176007833E2F5821230920276
:02317F0031FB22
:0C31810090F76EE0FAA3E07833EAF21257
:05318D0030B00231FB2F
:0C31920090F76DE0FA6005BA0A5F800E4D
:0E319E00758200123092758200123092804FBE
:0831AC00758200123092804789
:0931B40090F76DE0FA6002803E24
:0E31BD007582001230927582001230928030BE
:0A31CB0090F76DE0FABA20028005CB
:0531D500BA2123801067
:0831DA0078307407F2783174BB
:0831E200FCF20874F7F2801101
:0831EA00782D7407F2782A74B5
:0931F200FCF20874F7F208E4F2A3
:0B31FB0090DE0EE4F0782DE2602778F3
:0B320600297401F290DE117440F0907A
:0C321100F772E0FAA3E0FB782DE2FC7DF0
:0C321D0000C3EA9CEB9D5004782DEAF2FF
:03322900022F9DD4
:0A322C007830E2600C78297402F299
:0732360090DE117440F0224C
:0C323D0090F772E0FAA3E0FB4A600C7806
:0B324900297403F290DE117460F02283
:0B3254007829E4F290DE117448F022AB
:04325F007829E4F2F4
:07326300D20110AF02C2010D
:0A326A007827E2540160087827E29B
:0532740054FEF2800889
:0832790090F6F112184180E902
:0C328100A20192AF90DE0EE4F090DE118E
:0C328D00E0FA30E40A90DE117480F07862
:0332990029E4F233
:0C329C00EA30E20990DE11E4F07829E449
:0132A800F233
:0C32A9007829E2B4010BEA20E107C00222
:0532B500122F9DD00264
:0C32BA00EA30E0A57829E2B400028008A8
:0832C6007829E2B402978005AB
:0532CE001230D68090D3
:0C32D30012305390DE0EE4F07830E27010
:0C32DF000D7829E4F290DE117448F00232
:0232EB0032634C
:0932ED0090DE117440F00232631E
:0E32F60090DE0E7405F090DE11E0FA30E00874
:0833040090F76812184180EAFD
:01330C00229E
:0E330D0090DE0E7405F090DE11E04401F090A9
:0C331B00F768E0FAA3E0FB7825EAF2086E
:0A332700EBF290F768E4F0A3F02247
:05333100D310AF01C341
:09333600C0D07828E2700280206A
:0C333F0090F768E0FAA3E0FB4A700F78FA
:0C334B0025E2B4400708E2B40002800252
:023357008006EE
:063359001232F612330DE2
:05335F00D0D092AF2266
:05336400D310AF01C30E
:0B336900C0D0AA827828E27002802900
:0D337400C0021232F6D00290DE2AEAF0907C
:0E338100F768E02401F0A3E03400F090F76854
:0E338F00E0FAA3E0FBBA4006BB000312330DC8
:05339D00D0D092AF2228
:0E33A20090F76AE0FAA3E0FB4A704290DE0E5C
:0E33B0007404F090DE14E0FA20E00490FFFFB9
:0133BE0022EC
:0E33BF0090DE17E0FB7A0090DE16E0FC7D0049
:0E33CD004202ED420390F76AEAF0A3EBF0EA49
:0E33DB004B701190DE0E7404F090DE14E0547E
:0633E900FEF090FFFF2240
:0D33EF0090F76AE024FFFAA3E034FFFB90A2
:0D33FC00F76AEAF0A3EBF090DE28E0FA900B
:0E340900F76AE0FBA3E0FC4B700E90DE0E7441
:0A34170004F090DE14E0FB54FEF018
:073421007B008A828B8322ED
:02342800C2AF31
:0E342A001233A2AA82AB838A048B05BAFF0B71
:0B343800BBFF0890F3BB12184180E7B7
:05344300D2AF8C8222D3
:0D34480043BE801230B0122F0F439A029045
:0D345500DE06E4F090DE04F090DE02F022CE
:0E34620090DE07E4F090DE09F090DE0BF053F0
:0E3470009AFD90DE06E4F090DE04F090DE029D
:05347E00F053BE7F22A7
:0834830012344874B6C0E07475
:08348B0047C0E0745FC0E0746B
:0734930032C0E090F6F112D7
:0C349A00161DE58124FCF5817431C0E0B2
:0934A6007433C0E07464C0E074EA
:0734AF0033C0E09033A212CC
:0934B60015A5E58124FCF5812235
:0447B60075736200B5
:0748290000C20100000008BD
:0234BF00C2AF9A
:0E34C100122C9BAA82AB838A048B05BAFF28CB
:0D34CF00BBFF259000011218B890F6AC125A
:0D34DC001841AA828A047D00C004C00512B8
:0E34E9001904D005D004EC4D60CE7CFF7DFFB1
:0734F700D2AF8C828D83220D
:0434FE007A007B00D5
:0E350200C0031234BFAC82AD83D0038C068DA3
:0935100007BCFF05BDFF02802687
:03351900BB1000E4
:0C351C0050138B040B8B02EC2475F5821D
:09352800E434F7F5838E04ECF0A5
:08353100BE0D05BF000280067B
:06353900BE0AC6BF00C37C
:02353F008B02FD
:03354100BB1000BC
:0C35440050118B040BEC2475F582E4346C
:07355000F7F583E4F080EAC7
:033557008A822243
:08355A001234FEE58270F92233
:0C356200AA82C2D575F007E52C30E70402
:04356E00B2D5F404DA
:0E357200A430D50AF42401C5F0F43400C5F0ED
:0A35800024ADFB74F335F0FC740673
:0A358A002BF582E43CF583EAF02201
:09359400122CCE90000102191165
:05359D001234FE754F21
:0335A200BA7550A7
:0535A50047755180751F
:0635AA005202E4F553900B
:0E35B000F77575F000123881E5828583F045CD
:0735BE00F070047582012288
:0435C500754FBD750C
:0335C900504775F3
:0735CC005180755205E4F582
:0835D3005390F77575F000122A
:0E35DB003881E5828583F045F070047582FF2B
:0135E90022BF
:0935EA0090F775E070ADF5822246
:0435F300AA82AB837A
:0E35F7008A828B83E493FCA3AA82AB83ECFD53
:0E360500600F8D82C002C003123594D003D036
:033613000280E151
:013616002291
:0E361700AA82AB83C002C00312355AD003D082
:0B362500028A828B831235F302359D70
:0C3630007A357B007C409047C3C002C08C
:0E363C0003C0041235F3D004D003D0021ABA32
:03364A00FF011B62
:0E364D008A828B838CF0E41239001ABAFF01D6
:01365B001B53
:0E365C008A828B838CF0740D1239009000A4CA
:07366A00E493FD740193FEDF
:053671001ABAFF011B65
:0A367600754F0AE4F5508D828E8333
:0E368000C002C003C004C005C006124052AF15
:0E368E0082D006D005D004D003D00274302FB5
:0C369C008A828B838CF0123900754F0A73
:0C36A800E4F5508D828E83C002C003C088
:0E36B40004124088AF82A883D004D003D00255
:0836C2008F058806EF4870A790
:0E36CA008A828B838CF0124036FDA3AA82AB5D
:0E36D80083EDFE60138E82C002C003C0041298
:0A36E6003594D004D003D00280DA3E
:0336F00002359D03
:0736F300122D49122D259054
:0636FA0047CF12361790C5
:0E37000047DB123617AA82BA01047582012235
:04370E00758200229E
:07371200D20210AF02C20257
:0D37190030970A90F774E4F0438C028009A9
:0937260090F7747401F0538CFD5E
:05372F00A20292AF228E
:0637340090012C12191196
:0E373A007582031236F3E582701E9000641251
:0D37480019117582021236F3E582600690B9
:0537550047DF123617EA
:08375A0090006412191180D8DF
:073762009047E512361790B5
:0637690047EB12361712B7
:06376F0036309047F11214
:0C3775003617E4C0E0C0E074CEC0E07481
:073781002CC0E0902C9B120C
:0C37880015A585822CE58124FCF58175D7
:083794008200123562123712A7
:0B379C0090F774E0FA700890F77412C8
:0437A700184180F154
:0E37AB0090F774E0FA60EA7402C0E0E4C0E057
:0E37B90075820212221F1581158190012C12BB
:0437C700191180E074
:0C37CB00C022C0E0C0F0C082C083C00279
:0E37D700C003C004C005C006C007C000C0018A
:0D37E500C0D075D000C2EBE58A30E70912B4
:0637F200371290F774127B
:0237F800187F38
:0E37FA00758A00D0D0D001D000D007D006D004
:0E38080005D004D003D002D083D082D0F0D0FF
:04381600E0D02232AA
:0E381A00122D76758202122D49C29643FE4091
:0D38280053FE7F43F680439A10438D807459
:08383500F7C0E07447C0E07425
:08383D0034C0E07437C0E090D4
:0C384500F78512161DE58124FCF5812298
:0347BA004F4B0062
:0647BD004552524F52006C
:0C47C30041544E3D54656C6542542D007D
:0C47CF000D415445300D415451300D0097
:0447DB0041540D0038
:0647DF0041544C340D00B2
:0647E500415445300D00B7
:0647EB00415443310D00B2
:0647F100415451310D009E
:0347F700627400E9
:0400000002014D327A
:03000B00021F3899
:0100130032BA
:03001B00022B5263
:0100230032AA
:01002B0032A2
:03003300022F2277
:01003B003292
:0300430002217324
:03004B00022E4C36
:01005300327A
:01005B003272
:01006300326A
:01006B003262
:03007300022C114B
:03007B000237CB7E
:03008300022678DA
:0301A900020086CB
:0500860012385180FE5C
:0D385100122EE075820312224275820112D0
:06385E0021EE122EB21251
:06386400084C123483122F
:06386A0012AC122B121239
:0638700026721220041272
:06387600381A121F1312A4
:05387C000D0A0219B560
:0847FA00312E36000000000022
:0E480200616C7475736D657472756D2E6F72D6
:0248100067003F
:0C48120054656C6542542D76312E300048
:0E00AA001201100102000020FEFF0E000001F6
:0E00B8000102030109024300020100C03209E7
:0E00C6000400000102020100052400100105E3
:0E00D400240101010424020205240600010794
:0E00E2000581030800FF09040100020A000066
:0E00F0000007050402400000070585024000DD
:0E00FE000004030904200361006C0074007507
:0E010C000073006D0065007400720075006DD8
:0E011A00002E006F007200670018035400658D
:0E012800006C006500420054002D007600318E
:0E013600002E0030000E03300030003000308C
:0601440000300031000054
:0A388100AA82AB83ACF0E552455378
:06388B0070049000002211
:05389100AD4FAE50AF89
:0438960051A852A93A
:01389A0053DA
:05389B0018B8FF01193F
:0E38A000E84960368A828B838CF0124036F540
:0C38AE00546029C000C0018D828E838F01
:0A38BA00F0124036F8B55402800603
:0638C400D001D0008010CD
:0938CA00D001D0000ABA00010B84
:0738D3000DBD00C40E80C111
:0E38DA008A828B838CF0124036FA3395E0FB25
:0E38E8008D828E838FF0124036FD3395E0FC0A
:0A38F600EAC39DF582EB9CF58322E6
:06017C00E478FEF6D8FD58
:08015A007907E94400601B7AFB
:0501620001904829781E
:03016700FC759391
:0A016A00F7E493F2A308B8000205C1
:0801740093D9F4DAF27593FF50
:0E39000020F71030F6118883A88220F507F614
:05390E00A88375830091
:013913002291
:03391400F280F747
:02391700F0229C
:08391900E54F455060467A01BC
:07392100E54F25E0F54FE53D
:0939280050334012F550E5829580
:0A3931004FE583955040030A80E63D
:03393B00C3E55091
:07393E0013F550E54F13F5EE
:013945004F32
:0A394600C3E582954FF5F0E5839587
:08395000504005F58385F0826B
:07395800C3E55013F550E533
:06395F004F13F54FDAE101
:01396500223F
:0C396600AAF0FBE582854FF0A4FCADF058
:0C397200E583854FF0A42DFDE435F0FE48
:0C397E00E5828550F0A42DFDE5F03EFE32
:0C398A00E433FFEA854FF0A42EFEE5F0C8
:0C3996003FFFE5838550F0A42EFEE5F015
:0C39A2003FFFE5828551F0A42EFEE5F009
:0B39AE003FFFEB854FF0A42FFFEA85E0
:0A39B90050F0A42FFFE5838551F0C4
:0C39C300A42FFFE5828552F0A42F8EF0A7
:0539CF008D838C8222B3
:080182007834E84400600A79BA
:03018A000075936A
:06018D00F0E4F309D8FCC8
:0801930078C8E84407600C790C
:0B019B000890F034E4F0A3D8FCD9FA7F
:0539D4007A10E4FBFC89
:0E39D900E58225E0F582E58333F583EB33FBD1
:0A39E700EC33FCEB954FF5F0EC9586
:0939F100504006FCABF0438201DA
:0339FA00DADD22F1
:0A39FD00AA82AB83ACF07D007E00CF
:0E3A07008A828B838CF0124036FF60258F82FE
:053A15000ABA00010BDC
:0E3A1A00C002C003C004C005C00612149FD035
:0E3A280006D005D004D003D0020DBD00D20E92
:023A360080CF3F
:0E3A380075820AC005C00612149FD006D00584
:063A46008D828E83A32295
:02008B00E4731C
:063A4C00C01F85811F125E
:053A5200149FD01F22AB
:083A570085824585834685F058
:053A5F0047E4F542F50B
:043A640043F544855D
:033A68003548904E
:053A6B003A4C023B3063
:063A7000C01F85811FE567
:073A76001F24FBF548E4F5F5
:043A7D0042F543F5D6
:073A810044E51F24FBF88659
:063A880045088646088691
:053A8E0047903A4C12C4
:053A93003B30D01F22B2
:073A9800AA82C038C039C04A
:063A9F003A74AFC0E074B0
:063AA5003AC0E0C036C08B
:043AAB00378A8222B2
:0A3AAF001581158115810540E4B56D
:043AB9004002054181
:013ABD0022E6
:0E3ABE00AA8274302AFA24C6500A74072AFA23
:063ACC0030030343022059
:053AD2008A82023A980F
:0E3AD700E582FAC4540FF582C002123ABED046
:093AE50002740F5AF582023ABE88
:063AEE0085824FAB3BACEA
:043AF4003CAD3DAEFA
:043AF8003EAF3F7529
:023AFC00502058
:0E3AFE00EF2FFFEE235401FA4207EB2BFBECF7
:0C3B0C0033FCED33FDEE33FEC3EF954FAC
:0A3B18004008EFC3954FFF4303017F
:063B2200D550D98B3B8C4D
:043B28003C8D3D8E05
:043B2C003E8F3F2267
:073B3000858236858337858D
:033B37004238858C
:033B3A0043398587
:043B3D00443AE4F52D
:033B410040F5410B
:053B4400AA45AB46ACF0
:0C3B4900478A828B838CF0124036FD749A
:093B5500012AF545E43BF5468C1C
:083B5E0047EDFA700302401765
:053B6600BA25028003F6
:033B6B0002400F06
:053B6E00C204C205C203
:043B730006C207C2BD
:043B770008C209C2B5
:043B7B000AC20B75FA
:083B7F004900754A007DFFAE0C
:043B870045AF46AB55
:013B8B0047F2
:0E3B8C008E828F838BF0124036FAA3AE82AF8A
:063B9A00838E458F468B6F
:0B3BA00047BA25078A82123A988099E4
:053BAB008A04BC30009B
:0D3BB000402A8A04EC24C64023BDFF13E523
:0B3BBD004A75F00AA4FCEA24D02CF5A5
:073BC8004A70C1D20580BD67
:0D3BCF00ED75F00AA4FCEA24D02CFD80B0B6
:0A3BDC00BA2E07BDFFAA7D0080A6E7
:053BE6008A04BC61002F
:0D3BEB00400E8A04EC248540075302DFD20F
:033BF80003800245
:023BFB00C20303
:053BFD00BA2002805512
:053C0200BA2B02804B0B
:053C0700BA2D0280410E
:053C0C00BA4202804BEA
:053C1100BA43028050DF
:063C1600BA4403023DC1A7
:063C1C00BA4603023DD789
:063C2200BA4903023DC196
:053C2800BA4C028034DB
:063C2D00BA4F03023DC87E
:063C3300BA5003023D58E7
:053C3900BA5302804CAB
:063C3E00BA5503023DCD62
:063C4400BA5803023DD254
:033C4A00023DDB5D
:053C4D00D204023B8CD3
:053C5200D206023B8CCC
:053C5700D207023B8CC6
:053C5C00D209023B8CBF
:053C6100D20A023B8CB9
:083C660030090AE54814F88852
:053C6E00488602800FF2
:0A3C7300E54824FEF888488603089F
:053C7D008604188B0213
:083C82008A82123A98023DE427
:0A3C8A00E54824FDF8884886030889
:0A3C9400860408860618188B3B8C86
:043C9E003C8E3D8596
:063CA2003B82853C838596
:0C3CA8003DF0C00512401EAB82AC83D082
:063CB40005BDFF028B05B7
:0A3CBA0020042CC3EB954A5026E5C8
:063CC4004AC39BF54AAC67
:013CCA004AAF
:0C3CCB008C061C8C4AEE6014758220C030
:0E3CD70003C004C005123A98D005D004D003F3
:023CE50080E479
:023CE7008C4A05
:023CE9008D0448
:073CEB00853B82853C8385C7
:0C3CF2003DF0124036FDFA602F8C051CDE
:0E3CFE00C374808DF063F08095F050208A82B0
:0C3D0C00C003C004123A98D004D003ADEC
:043D18003BAE3CAFD3
:063D1C003D0DBD00010E8B
:053D22008D3B8E3C8F7B
:033D27003D80C11B
:063D2A00200403023DE449
:093D3000C3EB954A4003023DE497
:073D3900E54AC39BF54AAC0B
:013D40004A38
:0B3D41008C051C8C4AED7003023DE273
:0C3D4C00758220C004123A98D00480E96F
:0A3D5800E54824FDF88848860508B8
:0A3D6200860608860718188D3B8EB0
:043D6C003C8F3DAD9E
:043D70003DBD8000D5
:063D740040047A438014B4
:033D7A00BD600029
:063D7D0040047A50800BA7
:033D8300BD400040
:063D860040047A498002AE
:023D8C007A5863
:0E3D8E008A82C002123A9875823A123A9875EB
:0E3D9C008230123A98758278123A98D002BAA4
:043DAA004902800B3F
:053DAE00BA500280067E
:063DB300853C82123AD7A4
:083DB900853B82123AD78023FA
:073DC100D20875490A801CBD
:053DC800754908801799
:053DCD0075490A801297
:053DD200754910800D91
:043DD700D20B800982
:073DDB008A82123A9880026F
:023DE2008C4A09
:093DE400300B5AE54824FCF88874
:0C3DED004886040886050886060886073C
:083DF9001818188C3B8D3C8E5C
:043E01003D8F3E753E
:033E05003B1E75EC
:033E08003C4875BE
:023E0B003D80F8
:043E0D00853B4C8520
:033E11003C4D85A0
:053E14003D4E74012584
:073E19004CFFE4354DFCAD48
:043E20004E8F3B8CFA
:043E24003C8D3D850F
:063E28004C82854D8385EC
:0A3E2E004EF0124036FCFA70030259
:023E38003B4409
:073E3A008A82123A9880CC45
:073E4100E5497003023B4458
:043E4800754B5A302C
:073E4C00092BE54814F8887A
:0A3E530048E6FD3395E0FEFFFC8D0C
:043E5D003B8E3C8FCD
:043E61003D8C3E2036
:0A3E6500085EAC3B7D007E007F008C
:053E6F008C3B8D3C8E30
:053E74003D8F3E804C73
:093E7900300A1FE54824FCF8881A
:0C3E8200488604088605088606088607A6
:083E8E001818188C3B8D3C8EC6
:053E96003D8F3E802A73
:0A3E9B00E54824FEF8884886040874
:0C3EA500860518ED3395E0FEFF8C3B8D88
:043EB1003C8E3D8F77
:053EB5003E20080CACEA
:083EBA003BAD3C7E007F008E51
:033EC2003D8F3EF3
:0A3EC500300822E53E30E71BC3E49D
:093ECF00953BFCE4953CFDE495F3
:073ED8003DFEE4953EFF8C66
:043EDF003B8D3C8E4D
:053EE3003D8F3E80024E
:023EE800C2080E
:063EEA00D20CA84B7C0085
:0A3EF000753F00854982C004C00040
:0B3EFA00123AEED000D004200C0DE5C1
:0A3F05003FC4FDE6FE4DF618884BA0
:023F0F0080022E
:023F1100A63FC9
:083F13000C8C03B20CE53B45E8
:043F1B003C453D459F
:083F1F003E70CE884B8C03E5D7
:063F27004A7003754A0117
:0A3F2D00200524200421EB04FCAD64
:013F37004A3F
:0E3F3800C3EC9D5015758220C003C004C00567
:0C3F4600123A98D005D004D0031D80E68C
:023F52008D4A96
:0C3F540030080E75822DC003123A98D080
:053F600003154A802357
:0C3F6500EB602030060E75822BC00312AA
:083F71003A98D003154A800FB5
:0C3F790030070C758220C003123A98D06B
:033F850003154AD7
:053F8800200424AC4AF6
:0B3F8D008C051C8C4AC3EB9D502B30B0
:063F980005047D308002EB
:023F9E007D2084
:0E3FA0008D82C003C004123A98D004D0038072
:013FAE00DE34
:0A3FAF00C3EB954A5008E54AC39B96
:043FB900F54A80073E
:053FBD00754A008002BE
:023FC2008C4A27
:023FC400A84B08
:0A3FC6008B041BEC6026B20C200CEB
:0B3FD0000A08E6C4540FFC8C3F800779
:073FDB008604740F5CF53F42
:0C3FE200853F82C003C000123ABED00030
:043FEE00D00380D4A8
:063FF200200403023B4421
:023FF800AB4AD2
:093FFA008B041BEC7003023B4434
:0C400300758220C003123A98D00380EBB5
:08400F008A82123A98023B4438
:0740170085408285418322F0
:0B481E003C4E4F20464C4F41543E00E2
:04401E00AA82AB8344
:084022001240366003A380F890
:0C402A00C3E5829AF582E5839BF58322B2
:03014D0075815A5F
:0A0150001240C0E582600302008641
:0E40360020F71430F6148883A88220F507E6E0
:06404400A8837583002231
:03404A00E280F71A
:03404D00E49322D7
:02405000E0226C
:0E405200C2D5E58330E70DD2D5E4C39582F5E3
:0640600082E49583F58364
:0A406600E55030E70BE4C3954FF579
:054070004FE49550F53E
:0140750050FA
:0E40760012391930D50BE4C39582F582E4951A
:0340840083F5833E
:014087002216
:0E408800C2D5E58330E70DD2D5E4C39582F5AD
:0640960082E49583F5832E
:0A409C00E55030E70DB2D5E4C395FE
:0540A6004FF54FE49509
:0340AB0050F5507D
:0E40AE001239D430D50BE4C39582F582E49527
:0340BC0083F58306
:0140BF0022DE
:0440C00075820022E3
:00000001FF
